:100000009A28B800841780048413A201201CA2003F
:1000100010200319952810200319952810209528E1
:100020003808A2060130A000A10100083805220608
:10003000031D0800A00A0319A10F15280800A60037
:100040003A0884000930A70003102B20A60CA70B48
:10005000252803142B288413B71D3A2800083804D8
:10006000371D38068000841700083804031C380642
:100070008000452800083804031C38063719380664
:1000800080008417380980054528370D0639A000FF
:100090004E20A100A00A4E2000006E2800308A00E9
:1000A00020088207013475340334153400343C349D
:1000B0000C34D9348001840AFF3E031D5A28952848
:1000C000A301A200FF30A207031CA307031C95286D
:1000D0000330A100DF306E206228A101E83EA000BD
:1000E000A109FC30031C7728A00703187428A00777
:1000F0006400A10F742820187D28A01C812800000E
:1001000081280800A20003308528A80023082102C6
:10011000031D8C2822082002043003180130031923
:1001200002302805031DFF30952883130313831223
:1001300064000800FF2383169000831207309900A3
:1001400083169F01103085008312850120308400C2
:1001500040305A20A00105308400103001202008D2
:10016000BC002108BD003C08A0003D08A100A3017F
:10017000C8308220031DBD28AA280130D7006400A2
:100180000D3057020318D828A00105308400103024
:1001900001202008B2002108B3000310570D3C3E97
:1001A000840032088000840A33088000D70FBF28FB
:1001B0003E08A0003F08A100A30164308220031D77
:1001C000E3285610E42856144008A0004108A10076
:1001D000A30164308220031DEF28D610F028D61426
:1001E0004208A0004308A100A30164308220031D3F
:1001F000FB285611FC2856154408A0004508A1000C
:10020000A30164308220031D0729D6110829D615C1
:100210004608A0004708A100A30164308220031D06
:1002200013295612142956164808A0004908A1009F
:10023000A30164308220031D1F29D6122029D6165F
:100240004A08A0004B08A100A30164308220031DCE
:100250002B2956132C2956174C08A0004D08A10035
:10026000A30164308220031D3729D6133829D617FD
:100270006400D61B3C29D60A640056080A3C031DBC
:100280004229D6010530BA000130B8000230B7006B
:0A02900056081F2064306020AA28E1
:02400E00D43F9D
:00000001FF
